:1000000002006DFFFFFFFFFFFFFFFF90B61012140D
:10001000A4801E90B6181214A4801690B620121454
:10002000A4800E10981B32FFFFFFFF90B628121419
:10003000A412161F7CC812139890012DC082C08391
:1000400032C0E0C0D0E599B41B02D26E20740254D5
:100050007FC090439006C2D3D2D4C0A075A010F246
:10006000D0A0D09043902808D0D0D0E0327581A0A5
:100070007590FF75B0FF75A800758911758850756A
:100080002C00C29875B810C294C26978FFE4F6D803
:10009000FD7E06758B21758DA6C28F121A37121A36
:1000A00005308FF7C28FDEEB7598587587807455D1
:1000B0007895C6B45527F47896C6B4AA028006B4DB
:1000C000551B1207651200CB02012D121A051207EB
:1000D0007175100075110012056EC26E2211CBD21F
:1000E0006CD27612148FE4F513F52D750901120701
:1000F0004C121E6B1205C5C27BD27612148F742A65
:10010000121442C276752F08D27FD27DB2630201EB
:1001100047751000751100901FA1121503D27B7C4A
:10012000321213988007743F121465D26975D0009B
:100130007581A0750A8112022C750A8C12022C306E
:100140007B057C641213AA75D0007581A012148FF0
:10015000745E306302742A121958800312148F746B
:100160002AC26012185C307A07D276741A121442CE
:10017000C276C26A12161F30690312161F438850D6
:10018000D2B5C2B510662CC27675D0007581A0C2FA
:100190006CD26B1217EA70181218D360EA1215E7C6
:1001A00020690930630224109001BD93FE20E72DE1
:1001B0000203447C6412139874500203444F554E5A
:1001C00053594C80485C5A45415B54514043564E0C
:1001D00053474C44524B4A5742504A584620E00538
:1001E000120518212D0200C29001F01212E3212DF8
:1001F00002B602FE015C02F2033E032C032F03321F
:1002000002C6030102BB02EF015C030803350310C1
:10021000015C015C02DB025503230326015C031829
:100220000338032902F5033B22750A87E513B40757
:100230000050149002390212E36214883090DC21DD
:100240000AA33B99D8A21C90B6301214A4E513124D
:10025000140802015C1207A3AA13C00212029F51E4
:1002600029E50AD0027014C00212159DD00220693F
:100270000514F5138005B42010AA130513E513B473
:10028000070040D675130080D1B40D0EC0131207BD
:10029000BCD013750A53512C212D12161F80BBEAB6
:1002A000B513028010C0138A13750A82512CD01323
:1002B000750A81512C22307B20B27E020AE3D27A69
:1002C0008006C27A8002B27A207A0790B63712147A
:1002D000A42290B6401214A422212D021693207F4E
:1002E000012212161F90200B1214A4215C21260259
:1002F0000DAF020A10307F030202E2020AD5020C9F
:100300009CE52F54BF02030C7440452FF52F21802C
:1003100002084F120518212DE50A600675140075B4
:100320003A0022020DF8020FEA02082802084202EF
:100330000D090205EB020DC6020868020B61020BF3
:10034000CA020D84F50AB45C0280F6B443107890BA
:10035000E65409B40908750A88512C02012DE50AF2
:10036000B41003020437B42F02803B54DFB45B01A6
:10037000D35031B44000402CC39440121D20B40A25
:10038000028003532FEFB41303120255C00A7450B6
:10039000B50A031202DE512CE50AD00AB50A05C3DC
:1003A000944031E8212D1217E4FFBF4205120518D1
:1003B000212DB43100400BB43801D350051215E79C
:1003C000F518BF430451BE212DBF452212151C90C4
:1003D000F004439006758A21758CA6C28DF0308D8D
:1003E000FC90B651600390B649121503215CBF52D0
:1003F00002016DBF540451C2212DBF4C02D27FBFF8
:100400005502C27FBF4D05E515121437BF530302D5
:100410000D84BF50028020BF571B12153A20690A75
:10042000306103121BBEF53F212DE53F3061031201
:100430001BAB121437212D20616FE509B40401D3E1
:10044000400412161FE4F509700890B65A1214A45D
:10045000802AB4010890B6631214A4801FB4020865
:1004600090B66C1214A48014B4030890B6751214DC
:10047000A48009B4040690B67E1214A412148F123C
:10048000159D206904F50980AEB42004050980A7F4
:10049000E509B404127C641213AAC27F90B68712D5
:1004A00014A47C32121398212DE509B40301D34022
:1004B0000412161FE4F509700890B6901214A48077
:1004C0001FB4010890B6991214A48014B4020890C5
:1004D000205C1214A48009B4030690B6A21214A4DE
:1004E00012148F12159D206904F50980BCB42004F4
:1004F000050980B5E509B403127C641213AAC27F12
:1005000090B6AA1214A47C32121398B401087CC8C5
:100510001213AA120B89212D1205B3750E86E52E32
:1005200012140812185A750E8612153AF5F0306931
:100530001EB42029E52E04F5F0540FB40B01D3406E
:100540000353F0F085F02E307BCE12056E80C95437
:100550000FB40B01D3503D85F02E120765789676C7
:100560005520693076AA1205B37C3212139875A80B
:1005700090E52E540FB40B01D34002740575C834B6
:10058000C0E090059B1212F0D0E08582CA8583CB33
:10059000C295C29875100075110022F3BBF700FBDD
:1005A00080FDC0FEE0FF70FFB8FFDCFFEEFFF7FF4D
:1005B000FAFFFDE52E540FC0E090B6B31212F0D052
:1005C000E01214A422C0137513071513120229E5B3
:1005D0000A700CD0E0C013750A80512C1207A3E5F5
:1005E0001370E7D013750A81512C22C01AC01BC0AA
:1005F0001CC01DC01EC01F1216937CC81213AA85F2
:100600001D31851E32851F33C5312401C531500A85
:10061000C5322401C5325002053374447F331216AB
:100620009E30690D547FB4200280060206D802066F
:10063000F690B7061214A4E51DC3951AF52BE51E16
:10064000951B422BE51F951C452B40DFE51AC395F2
:1006500031F52BE51B9532422BE51C9533452B706C
:1006600001D350CAC01DC01EC01FC51DC3951AC5E9
:100670001DC51E951BC51EC51F951CF51F451E4596
:100680001DC531251DC531C532351EC532C53335B1
:100690001FC533D01FD01ED01D851D54851E558506
:1006A0001F56121D3D85343530932D121D59E51D01
:1006B000B51A0DE51EB51B08E51FB51C030206E7BC
:1006C000121DD9C3C51D9401C51D500AC51E940035
:1006D000C51E5002151F80C1D01FD01ED01DD01CBA
:1006E000D01BD01A020111D01FD01ED01DD01CD09B
:1006F0001BD01A02012D851A54851B55851C5612D4
:100700001D3D8534353093D0121D59E51DB51A0DA8
:10071000E51EB51B08E51FB51C030206E7C531241D
:1007200001C531500AC5322401C53250020533C516
:100730001A2401C51A500AC51B2401C51B50020505
:100740001C80B390B70E12179502015CD276C27B63
:1007500012149290B7351214F190B72E1217957C9F
:100760002812139822C0D01207EFE6F2D8FCD0D09E
:1007700022E4752E37F51AF51BF51C751DFF751E45
:100780007FF51FF53EF536F537F538F539F53BF5CC
:100790003CF53D753F10751801F50BF514F53A78E9
:1007A000FFF622758216E5132408F583439006A808
:1007B00082E6F01207D570F7E509F022758216E59A
:1007C000132408F583439006A882E0F61207D5703B
:1007D000F7E0F50922A3E582B42B004008B45901E3
:1007E000D350027459B480027498F58264A02278C0
:1007F0007F75A00043900653D0E722C03E7CC8120C
:1008000013AAE53E601112081D30930B7C6412138D
:1008100098D53EF212081D3093FDD03E2290202341
:10082000121503E53E02147E9020231214A4E53E27
:1008300012140812185A750E8612153A206902F51C
:100840003E221207FB7F397E807D081216C22220CD
:100850007B001207FB12148F9020151214A47D0444
:100860007F3C7E841216C52212148FE533121410B9
:1008700079321215BA12185A1217153061158531CE
:1008800040853241853342121A6D854031854132AF
:100890008542330209DC750E85743D121465121D04
:1008A0002A12140512185A750E8620610512153A7F
:1008B000800312159DF5352069030209BAB420039F
:1008C0000209D4B44C03020DF1B40806121DD9027A
:1008D00009DCB44E12121DED121D3D853435633511
:1008E000FF121D620209DCB449107900E7F53512E8
:1008F0001D59121D93D9F50209DCB4592390B7484C
:100900001214A4750E83121D3412153A30690302B5
:1009100009B9855482855583C292121C890209DC6B
:10092000B4582390B74E1214A4750E83121D3412BE
:10093000153A3069030209B9855482855583C292FC
:10094000121CD70209DCB45370A831A932AA3312A1
:10095000161F90B7541214A4307B057C32121398E2
:1009600090B75D1214A4750E8512153AF535121D57
:1009700034E06535603AA3E582B51D07E583B51E11
:10098000028003020971E065356025858231858327
:1009900032121D7E70D812161F90B7651214A43043
:1009A0007B057C32121398883189328A330209DC44
:1009B0008582318583320209DC22121DED121D620F
:1009C000C0E0121D3DD0F065F0C0E07CC81213AA53
:1009D000D0E07005121D937003120D7CC031C0323F
:1009E000C033306115853140853241853342121B59
:1009F0004B85403185413285423312148FE53312E5
:100A0000141079321215BAD033D032D03102089690
:100A100012148F90B76E1214A4E4F548F549121D14
:100A200034C5482548C54850020549A3E0C54825B6
:100A300048C54850020549E582B51D07E583B51E46
:100A4000028003020A2B858231858332121D7E705B
:100A5000CD9020641214A479491215BA02015C9059
:100A6000B7771214A4121316121D20E4F548F549A5
:100A7000121D340582D5820215831582A3E0F5F09C
:100A80007808E4A2F092E1654823236548232365B2
:100A900048236549A2E6E54833F548E54933F54979
:100AA000E5F023F5F0D8DBE582B51D07E583B51E3B
:100AB000028003020A7C858231858332121D7E709A
:100AC000AF9020681214A479491215BA12132F029C
:100AD000015C020B6D207FFA120B4F23F518120BED
:100AE0004F800053D0E71207FB12148F7455307FEC
:100AF00002744C121465744A2061077449307E02F6
:100B0000744D121465742A3061077449307D027483
:100B100053121465742A307C0274311214657443C4
:100B2000207A027454121465120B4F75F008A41247
:100B30001BABC0E0E5F01213EDD0E01213DF307B09
:100B40000D74647C0A1213AA309303D5E0F522E5F4
:100B50001870027401B40801D350F8121C19F5186A
:100B600022E52F20E30320E25E6480F52F207F1032
:100B700090B77F1214A4D2637C3212139802012D15
:100B800090200B1214A402015CE52F20E30320E265
:100B9000366420F52F207D1B901FD51214A47C1ED7
:100BA00012139890B7881214A47C32121398D2634F
:100BB00002012D901FD51214A47C1E1213989020B0
:100BC0000B1214A402015C020126121D2012159DB5
:100BD0002069115515F53312153A206907F5328051
:100BE00035020C9CB40D02802DB44C0280F3B4206D
:100BF0000DE53F23F53F121BAB1214088018B42FEC
:100C00000D12153A121BBEF53FD261020CAEC26145
:100C1000753F100201262061F21207FB7C6412135B
:100C2000AA121492C031C032C033E53312143F12FD
:100C300013D0120C96C2D5120C5CD033D032D03106
:100C4000D2D5120C96120C5C700122E53170D212D2
:100C50001A3712153AB40DC42220D503120C96751A
:100C60008AD8758CFFC28D308DFD121D2F20D505C1
:100C70001214378010B47F01D35005B42000500205
:100C8000742E121442121D7E600BE531853FF084F4
:100C9000E5F070C5F4227420121442221207FB12F0
:100CA0001D2F121442121D7E30930270F2227556CF
:100CB000007CC81213AA7E1412149285314085322A
:100CC00041121A49E541121437E5401214377420D5
:100CD000121442C03F853154853255121D3D121405
:100CE0003FC5312401C53150020532E531B51D083B
:100CF000E532B51E03020D06D53FDAD03FDEB9124C
:100D00001613B40DA922D03F22121D20901FA51248
:100D100014A4E518B40102800B750E8412153AF57F
:100D20003420695812153AF53520695012148F9005
:100D3000B7911214A4E518B40102801E121DFFC061
:100D400035853435121D62D035121D7E600B121DA3
:100D5000FF121D62121D7E70DC22121D59A3E535A3
:100D6000F0E582B51D07E583B51E028003020D5D27
:100D7000858231858332121D7E70DF2212161F7428
:100D80003F021465121D2090B7991214A4121D344D
:100D9000F535121D7E121D34121D62853435121D6B
:100DA000D9121D59121D93121D7E70E102012D9062
:100DB000B7A21214A4121D2AC4F535121D62121D09
:100DC0007E70F202012D90B7AA1214A4121D2AF40B
:100DD000F535121D62121D7E70F202012DF53512DD
:100DE0001DFF121D6285311D85321E85331F121DA8
:100DF00093D26012127B80E590B7B1121503E4F52F
:100E000044F545F546F533D26CC268207E0C020FDE
:100E100028121262FB12151CDBFB12127B547FB4EA
:100E200053F8C2D512127B547F754800B43901D3F0
:100E30004003020EB8C39430900E3E0212E30E112E
:100E40000E540E8B0E7D0E1A0E1A0E1A0EAA0EAA34
:100E50000EAAD2D5121262C39403FB120EE62069C9
:100E600013EB6003120EF41215A2F4B5485230D5FC
:100E7000A902012D90B7BA121503020EC812126210
:100E800024FBFB121262B53991800612126224FC17
:100E9000FB121262F533C3953CC53365386315FF09
:100EA00025156315FF60B4020E1A12126260C5FBAD
:100EB000121262DBFB02120490B7C3121503800802
:100EC00090B7CC1215038000D28C12161F7F6410CD
:100ED0008D071217EA70F680F6758A1E758CB8C2F7
:100EE0008DDFEC02015C12151CC3953BF532121527
:100EF0001CF5312212151CC0E0121DFFD035121D49
:100F0000620531E531700E0532E53270080533E5D2
:100F1000335515F533DB012270DA0211F62068082B
:100F2000120EF41215A2254812127B547FB43AF81F
:100F300012151CFBF548120EE6206948E54454F0F2
:100F40002531F531E5323545F53212151C60CEB448
:100F50000203020FB3B40103021204B40303020F2D
:100F600028B404028024B40503020F28B4C8121266
:100F700015A22548701190E000E531442043900609
:100F8000F0020F28020E74020EC0C001E515F4F93C
:100F900012151C6539C0E012151CF533C3953CC50C
:100FA00033653859F9D0E049C2686002D268D0018F
:100FB000020F2312151CC0E0C4540FC3953CF53337
:100FC000D0E078467600C4D67845F612151C7845F0
:100FD000C4D618F654F0C39536E5459537E5464531
:100FE00015540F95389268020F231207FB90B7D55E
:100FF000121503121D2085394785384685374585EA
:101000003644121492754800121113307E030211F7
:101010005D1212C8E5474546454545447027E51F22
:10102000253C700302109A1212D71212CE1212D758
:10103000E5335515253CC454F01214311212D21266
:1010400011E7021097E54770151212D71212CE124F
:1010500012D71210771210891211E702109712128C
:10106000D71212CE1212DDE547121431E5461214E2
:10107000311211E7021097E54554F0F9E546540F97
:10108000253C551539C4021431E54454F0F9E545C1
:10109000540F29C40214311212C8EA12143112106A
:1010A000DFE41214311211D83093051210E45017F6
:1010B0001212C8E4121431E4121431E4121431741F
:1010C000011214310211E770CEE54745464545450A
:1010D000446009E54604F54670020547021011E533
:1010E0003B0213D1AA3FE533E53245316023E531B8
:1010F000C3951DF52BE532951E422BE533951F4513
:101100002B7001D3500B121113E532253B4531C32F
:1011100022D322C01DC01EC01FAA3FE4F556F555BC
:101120008A541554C51DC39531C51DC51E9532C5BC
:101130001EC51F9533F51F451E451DE51DC395545E
:10114000F52BE51E9555422BE51F9556452B700155
:10115000D35003AA1D0AD01FD01ED01D22745312D3
:101160001442E5397020E51F7008E5384533453CE9
:10117000600A7432121442EA240480177431121483
:1011800042EA240380167433121442EA240512142E
:1011900031E539121431E5382533353C121431125A
:1011A00010DF1211D81210E430930250B0745312B1
:1011B00014427B37E539700A0BE5384533453C70FE
:1011C000010BEB12143F2403F45407FB1214311BE0
:1011D0001212D2DBFB0211E7C002121D2F121431D2
:1011E000121D93DAF5D002E4C548F4207E01041202
:1011F00014371214922290B7DC12150312161FD264
:101200008C020ECDC001C0027A53207E027A3AE5EC
:1012100009B40402D26612151C7928758A21758CCE
:10122000A6C28D1217EAB50218D002D001E4F54427
:10123000F545F546F533C268207E03020F30020EF5
:101240002270D6308DDDC28DD9D1121848753B0081
:10125000753C0043900690E000E4F0D002D001021B
:10126000012D1217E41215E7C4C0E01217E412159D
:10127000E7D00048C5482548C54822C269C006785D
:1012800032D28CE53E046005440AFE8002C28C75B1
:101290008A1E758CB8C28DE51065117020308DF7EF
:1012A000C28D309320D8E87832DEE420691490B7FC
:1012B000E312150312161F12161F02017D12180BDE
:1012C000C269D00622020111743A12144222E412B9
:1012D0001437E412143722740212143122740412E7
:1012E00014312223F52B0493C0E0E52B93C0E022B8
:1012F00023F52B0493C52B93F583852B8222C0F015
:10130000C000F5F078FF08E893C36005B5F0F7E892
:10131000D3D000D0F022D058D02BC000C001C002E2
:10132000C003C004C005C006C007C02BC05822D0EF
:1013300058D02BD007D006D005D004D003D002D08F
:1013400001D000C02BC05822D058D02BC000C00103
:10135000C002C003C02BC05822D058D02BD003D01D
:1013600002D001D000C02BC05822D003D002D0013F
:10137000D00022D058D02BC001C002C003C02BC067
:101380005822D058D02BD003D002D001C02BC05847
:1013900022D003D002D00122758A18758CDCC28D50
:1013A000D28C108D0280FBDCEF22758A79758CFC63
:1013B000C28DD28C108D0280FBDCEF22758A79758C
:1013C0008CFCC28D308DFDC28DD504F0D508ED2288
:1013D000E47832261214317831E6021431D277C023
:1013E000E0C41213EFD0E0C2771213EF22D27712CB
:1013F0001471307707B4300474208002C277121958
:1014000058307B3E22206108C0E0C4121410D0E0A6
:10141000121471121958307B2922C0027A0823C095
:10142000E05401121410D0E0DAF4D00222547F808C
:1014300011C5482548C548C0E0C412143FD0E01289
:101440001471C294207605D2952095FBA2E72074F2
:10145000024480F59992E73099FDC29922750E8079
:10146000121465743D207B05547F121442121958E2
:1014700022540FB40A0040022407243022E6C0E0C0
:10148000C4121471121958D0E012147102195820A4
:101490007B0EC0E0740A121442740D121442D0E0A4
:1014A000750E802212148F750E80E493A3600AC01B
:1014B000E0121465D0E030E7F11219BB22C00179C7
:1014C00000E99360040930E7F8E9D001220217959A
:1014D000307610C082C083307B031214CDD083D00D
:1014E000828003207BE712148FE493B42003A3804F
:1014F000F8E493A3600CC0E0547F121442D0E030B3
:10150000E7EF22750E80E493A3600AC0E012195839
:10151000D0E030E7F11219BB22D0F0221215E420FE
:101520006917C4C0F0C0E01215E4D0F02069EA45A4
:10153000F0D0F0C5482548C5482212159D20690DF8
:10154000C4C0E012159DD0F020690245F0221215AA
:101550003A206902F535221217F9B43000400CB474
:101560003901D35006C39430C26922D269221215C0
:101570005720691275F00AA4C0E0121557D0F02068
:10158000690425F0C2692212155720690FC4C0E012
:10159000121557D0F020690425F0C26922121613E3
:1015A00080451215E420690DC4C0E01215E4D0F0A6
:1015B00020690245F022C2D5800E1215BE19C2D58F
:1015C000E7C4121471121958E71214711219582035
:1015D0007B04E7121437221215DB19E7C00112143D
:1015E00037D001221217F9B43000401EB43901D3AC
:1015F000400AB441004013B44700500EC39430B4C5
:101600000A004003C39407C26922D269221217F963
:101610000215E7754A00207B030217F902186CC017
:10162000D053D0E7C006C0E07E02758A18758CDC06
:10163000C28D740EC296C296C296C296C29614709D
:10164000F3740ED296D296D296D296D2961470F3A6
:10165000108D0280DDDED3D0E0D006D0D02278021B
:10166000758A47758CF5C28D539069108D0280FB89
:10167000758A47758CF5C28D439096108D0280FB5C
:10168000D8DE22C296758AAA758CFFC28D308DFD78
:10169000D2962274537F1C12169E74467F1F12141A
:1016A0008F12145D7E827D051216C522C005C0060C
:1016B000C0077F337E807D051216C2D007D006D0CA
:1016C000052212148F121316C269EFF98E0EEDC3A4
:1016D000139262FAC002306205E712141019121553
:1016E000BE19DAFA098E0ED26B12185AD002C269EC
:1016F00030620512159DC0E020690312153AC0E062
:10170000DAF6EDC3133400FAD0E0206901F709DA04
:10171000F712132F22121373750E84121D20121547
:101720009D790120694EF533E4F531F532C533F585
:1017300031750E847884E6FA12159D206936FBEA2D
:101740007884C6C0E0121777D0E0750E841219585D
:10175000EBC442337404C5333303C533C53133C5D9
:1017600031C53233C532C53333C533D5E0E809B9A5
:10177000050040BD021391C00179077887E6C0E0FB
:1017800018D9FA7907750E80D0E0121958D9F912D4
:101790001958D00122750E80C082C083E493A32023
:1017A000E7166017121958E50EB480F07C32121358
:1017B000AAD083D082A380E0121958D083D082129D
:1017C00019BB22740A121442740D0214421217F447
:1017D00070271218D322E510651170031218C92260
:1017E000F512C294E510651160F61217F4700AF54F
:1017F00012C29422E510651122E5106511700C20CB
:1018000093F7751000751100020111C0D0439006C6
:10181000C2D3D2D4C0A075A010E3D0A009D0D020EC
:101820006006A2E5B0E692E5206C1020750D207BE5
:101830000A2095FDF5993099FDC299C27B22D0D03E
:1018400090B7EE1214A480FE75100075110022C02E
:10185000E012185AD0E0D5E0F6227420207B031263
:10186000144222207B05741012144222C000758A93
:1018700021758CA6C28D1218D37005108D0B80F6C1
:10188000306B03121958D000227897E6601506B421
:10189000151176141216837890E6137408400274BA
:1018A0002080DD758A21758CA6C28D054AE54AB473
:1018B0000A04742D800EB414B5754A00A80EE6B45F
:1018C0002D0274201219A280A512131612192312C8
:1018D000132F221213161219236044EDFB12192341
:1018E000EBB505F2121923EBB505EB209328121680
:1018F00083D27BEA47F7ED12B7F730E72230E608EC
:101900007890E630E30A7408547F78977601800F68
:1019100012132F02010C78977600EAF457F7E412BD
:10192000132F2279907DFF7FFF7A800FEA23CA3040
:10193000E30709B995F1E4801E1219C80DEA57C0F2
:10194000E0E9540FFCEF5407C44C1219D8E420937B
:1019500001EAD0046C60D422547FC0E0206A15E50F
:101960000EB48010C00078087420121983D8F9755D
:101970000E80D000D0E0B40D05750E80803DB420FF
:10198000004038C000A80EF6C0E01219A2050EE50E
:101990000EB48701D34003750E80D0E0D000221230
:1019A0001471C0E0E50E540FF41219CAD0E0A2E59C
:1019B000B0E692E51219D8D2B5C2B5C0E01219C886
:1019C00074201219D8D0E0227410D2B5C2B5C00468
:1019D0007C1EDCFE7C108004C0047C40C0E05C24E3
:1019E000FFC2B5C0A8C2AFD2B54002C2B5D0A8747C
:1019F000051470FDECC313FCD0E050E0C2B57C0FC1
:101A0000DCFED00422C0007878D2B5C2B5758ABB9E
:101A1000758CFFC28D308DFDD8EFD000C00078905E
:101A2000E4F608B895FBD000221219C874FF121909
:101A3000D8A293B3927B22C0F0750E807420121945
:101A400083E50EB480F6D0F02212134878107900A6
:101A50007A00C54033C540C54133C541E939D4F9A1
:101A6000EA3AD4FAD8EC89408A4102136AC000C02D
:101A700001C002121ABCC042E4C542781079277A2C
:101A800000121A97D0E0C478A079867A01121A97CA
:101A9000D000D001D00222540F30E00FC54028C53D
:101AA00040C54139C541C5423AC542CA3303CAC8D7
:101AB00033C8C933C9CA33CA0370DC22C0E0C000CE
:101AC000C001C041754100E540540FC540780A7916
:101AD00000C4121AF178647900D0E0C0E0121AF163
:101AE00078E87903D0E0C4121AF1D000D001D0E038
:101AF00022540F30E00AC54028C540C54139C541D0
:101B0000C93303C9C833C8C933C90370E422C00646
:101B10007E18E4F553F552F551F550E54033F540A4
:101B2000E54133F541E54233F542E5503550D4F512
:101B300050E5513551D4F551E5523552D4F552E5C1
:101B4000533553D4F553DED3D00622754300C0502D
:101B5000C051C052121B0E855040855141855242E2
:101B6000D052D051D05022C006750000750100C37C
:101B70007E10E54033F540E54133F541E50033F5AE
:101B800000E50133F501B54305E500B54200400F1E
:101B9000C3E5009542F500E5019543F5010540C315
:101BA000DED0850042850143D00622C00075F00AD0
:101BB00084A8F075F00A84C5F0C448D00022C0E0C3
:101BC000C4540F75F00AA4D0F053F00F25F022E5AD
:101BD000408542F0A4F54485F045E5418542F0A4F6
:101BE0002545F545E435F0F550E5408543F0A4255D
:101BF00045F545E5F03550F550E43400F551E54143
:101C00008543F0A42550F542E5F03551F5434542B2
:101C100024FF85444085454122600FC0007800C301
:101C2000083350FCE413D8FDD00022600FC00078C8
:101C300000C3081350FCE433D8FDD00022C006C016
:101C4000037E087B001350010BDEFAEBD003D006B5
:101C500022540FA2E375F000121C605002C5F0225E
:101C60005407048322010204081020408054070412
:101C70008322FEFDFBF7EFDFBF7F600CC00078FF23
:101C8000C3081350FCE8D000221213486046C082FB
:101C9000C083C040C041858240858341FB7A00C03B
:101CA00082C08378017900854082854183E05401B8
:101CB0006003E849F9A3E823F830E0F18582408524
:101CC0008341D083D082E9F00AA3DBD3D041D04056
:101CD000D083D08202136A1213486041C0A0C08230
:101CE000C08375A011FBFA7900E0C090439006F321
:101CF000D09009A3DBF37900D083D082C082C08367
:101D0000C090439006E3D090F8097B08E803C854DC
:101D100001F0A3DBF7DAE9D083D082D0A002136A06
:101D2000851A31851B32851C3322121DED800E125F
:101D30001DFF800985315485325585335643900601
:101D4000E5552514C0E0E556353A90C000F08554BD
:101D500082D083C292E0F534228531548532558594
:101D60003356E5552514C0E0E556353A90C000439A
:101D70009006F0855482D083C292E535F0223093EC
:101D800034E531B51D0DE532B51E08E533651F5547
:101D9000156021E5312401F531500EE43532F5327C
:101DA0005007E435335515F533853356853255855F
:101DB000315474FF22020111853154E532253BF57F
:101DC00055E533353CF55622853154E532C3953B14
:101DD000F555E533953CF55622C3C5319401C5311F
:101DE000500AC5329400C532500215332285315451
:101DF000E532C3953BF555E533953CF556800985AD
:101E00003154853255853356E51813500122851D0E
:101E100044851E45851F46C5442401C544500AC556
:101E2000452401C5455002054685542B305810F510
:101E30002BE5444254E5454255E5464256E52BC361
:101E4000C55613C556C55513C555C55413C554C3FA
:101E50001350D62212153A206910121533F532129A
:101E6000153A206905121533F53122D276E4F531A1
:101E7000F532F53343900690C000E533F0C292602E
:101E800002C291853283853182E0F87455F0E0B466
:101E90005526F4F0E0B4AA20E8F0E5822410F5829B
:101EA00050E70583458370E10533858231858332B0
:101EB000E533B40701D340BCE533F541E53254F0D6
:101EC000F5407802C5411323C541C54013C540C53F
:101ED0004113C541D8EE121A49740D121442750E01
:101EE00080C2D5E5411213EDE5401213DF744B12A9
:101EF0001465E53314F515750E8690B8101214AA02
:101F00007C6412139822C082C08390D03043900624
:101F1000F4F0D083D0822290D030439006F4F022A7
:101F200090D030439006121C60F02290D030439045
:101F300006121C6DF022439006E490F000F0A3F02E
:101F400090F002F0A3F022464149CC544553544945
:101F50004EC7434F5059494EC75645524946D94F2F
:101F6000564552435552AE2D5643C32D5650D0457B
:101F700052522E524E47D34552522E524E47C645CC
:101F800052522E4D4FC443414C2E5345D44C4F41D9
:101F90004420A3454D554C4154C553555350454ECF
:101FA000C4455849D444415441AD455252314D4144
:101FB00053CB455252324D4153CB4D49534B54B103
:101FC0004D49534B54B24D4953534BD4534543554C
:101FD0005245BF554E5345435552C550524F475237
:101FE00041CD4C4F432E20202050524F4D0A0D0022
:101FF000424C414ECB4255534552D24D49534F432B
:00000001FF
